:1008B8001201000200000040051603800100010239
:1008C80000010A06000200000040010009022000A1
:1008D800010100A0320904000002FF000000070522
:1008E8000202000200070586020002000902200039
:1008F800010100A0320904000002FF000000070502
:1009080001024000000705810240000004030904B9
:1009180026034100430043004500530020004900DE
:100928002F004F002000500072006F006400750017
:1009380063007400730016035500530042002D0035
:0E094800440049004F002D0039003600000029
:0A00360000010202030304040505A3
:10095600E4F50BF50AF509F508C203C200C202C2A6
:1009660001120CE87523087524B8752B08752CCA76
:100976007521087522D4752908752AF4752D09750F
:100986002E14D2E843D82090E668E04409F090E6B9
:100996005CE0443DF0D2AFD20412000390E680E062
:1009A60054F7F0C2033001051203CEC20130032909
:1009B6001200405024C203120D0E20001690E6824B
:1009C600E030E704E020E1EF90E682E030E604E084
:0E09D60020E0E4120C90120E0E120A7080C780
:1003CE0090E6B9E0700302047F1470030204FC246B
:1003DE00FE700302057F24FB700302047914700380
:1003EE00020473146073146076240560030205DF43
:1003FE00120E1040030205EB90E6BBE024FE6022D5
:10040E0014603324FD601114602224067048E52325
:10041E0090E6B3F0E5248037E52B90E6B3F0E52CBB
:10042E00802DE52590E6B3F0E5268023E52790E6BE
:10043E00B3F0E528801990E6BAE0FF120CBCAA06CC
:10044E00A9077B01EA494B600DEE90E6B3F0EF9001
:10045E00E6B4F00205EB0205E4120DE00205EB1224
:10046E000DFA0205EB120DF20205EB120DCE02058E
:10047E00EB120E1240030205EB90E6B8E0247F600B
:10048E001514601924027063A200E43325E0FFA264
:10049E0002E4334F8041E490E740F0803F90E6BCA9
:1004AE00E0547EFF7E00E0D394807C0040047D010A
:1004BE0080027D00EC4EFEED4F2436F58274003E38
:1004CE00F583E493FF3395E0FEEF24A1FFEE34E6CF
:1004DE008F82F583E0540190E740F0E4A3F090E6BC
:1004EE008AF090E68B7402F00205EB0205E4120E20
:1004FE001440030205EB90E6B8E024FE60162402D9
:10050E0060030205EB90E6BAE0B40105C2000205F5
:10051E00EB0205E490E6BAE0705590E6BCE0547E3E
:10052E00FF7E00E0D394807C0040047D0180027D3C
:10053E0000EC4EFEED4F2436F58274003EF583E45A
:10054E0093FF3395E0FEEF24A1FFEE34E68F82F5A4
:10055E0083E054FEF090E6BCE05480131313541F56
:10056E00FFE0540F2F90E683F0E04420F0806E8081
:10057E0065120E16506790E6B8E024FE601A24024B
:10058E00705B90E6BAE0B40104D200805090E6BAF7
:10059E00E0B402028047803E90E6BCE0547EFF7ECF
:1005AE0000E0D394807C0040047D0180027D00EC4D
:1005BE004EFEED4F2436F58274003EF583E493FF34
:1005CE003395E0FEEF24A1FFEE34E68F82F58380B3
:1005DE0008120056500790E6A0E04401F090E6A005
:0405EE00E04480F075
:0105F20022E6
:0300330002004E7A
:04004E0053D8EF3262
:04004600022F000085
:0407FC0043B12022C3
:040E0A0053B1DF22DF
:100CE80090E600E054E7F0E58E54F84405F58ED21E
:100CF80000120E027580FF7590FF75B2FF75B31F65
:060D080075B620020E0A80
:100A7000E5336035E530452F7006752F2F7530FF53
:100A8000E53015307002152FE530452F7004F53331
:100A9000800FAE2FAF307C0B7DFF12074AEF20E0B6
:100AA00005120E0A80031207FCE5B190E68020E7EC
:0A0AB00005E04408F022E054F7F0DE
:010ABA002219
:02004000C322D9
:020E0E00D322ED
:020E1000D322EB
:080DF20090E6BAE0F534D322CB
:100DCE0090E740E534F0E490E68AF090E68B04F08C
:020DDE00D3221E
:080DFA0090E6BAE0F531D322C6
:100DE00090E740E531F0E490E68AF090E68B04F07D
:020DF000D3220C
:020E1200D322E9
:020E1400D322E7
:020E1600D322E5
:1000560075330190E678E05410C4540F4450F532DD
:1000660013E433F53590E6B9E012079F00911000CE
:10007600ED11013A1201DB3001DB310245A20245E6
:10008600A3023FA90215AC000003CA90E6BEE090A9
:10009600E68BF090E6A0E020E1F9E4F512F51374A2
:1000A600402513F58274E73512F583E0FFE4251346
:1000B600F58274803512F583EFF074462513F582C8
:1000C60074E73512F583E0FF74082513F582748012
:1000D6003512F583EFF00513E51370020512640679
:1000E600451270BB0203CCE4F512F513E42513F5B3
:1000F6008274803512F583E0FF74402513F582740F
:10010600E73512F583EFF074082513F58274803510
:1001160012F583E0FF74462513F58274E73512F570
:1001260083EFF00513E5137002051264064512709D
:10013600BB02020590E6BEE090E68BF090E6A0E0FA
:1001460020E1F990E6BDE0FF90E6BCE04F701D901F
:10015600E6BAE05401C454F0FF90E74DE0F4540FC2
:100166004FF59090E74CE0F4F580801C90E74CE06A
:10017600F4FF90E74EE04FF58090E74DE0F4FF90F6
:10018600E74FE04F540FF590E4F512F51374402550
:1001960013F58274E73512F583E0FFE42513F58243
:1001A60074803512F583EFF074462513F58274E7F3
:1001B6003512F583E0FF74082513F5827480351235
:1001C600F583EFF00513E513700205126406451278
:1001D60070BB0203CC90E740E580F0A3E590F0A366
:1001E600E5A0F0A3E5B0F0E5B130E4047F018002BC
:1001F6007F0090E6BAEFF0E5B1540F90E744F0E4E3
:1002060090E68AF090E6BEE090E68BF00203CC9092
:10021600E6B5E054FEF090E6BFE090E68AF090E6A0
:10022600BEE090E68BF090E6BBE090E6B3F090E699
:10023600BAE090E6B4F00203CC7535014332019082
:10024600E6BAE0750C00F50DA3E0FEEE420C90E672
:10025600BEE0750E00F50FA3E0FEEE420E90E6B886
:10026600E064C06003020333E50F450E700302032A
:10027600CC90E6A0E020E1F9C3E50F9440E50E94AA
:10028600005008850E10850F118006751000751137
:100296004090E6B9E0B4A336E4F512F513C3E513CE
:1002A6009511E51295105060E50D2513F582E50CC4
:1002B6003512F583E0FF74402513F58274E7351295
:1002C600F583EFF00513E51370D3051280CFE4F53F
:1002D60012F513C3E5139511E512951050197440E4
:1002E6002513F58274E73512F58374CDF00513E511
:1002F6001370E0051280DCAD117AE779407F40ABE0
:1003060007AF0DAE0C120ABBE490E68AF090E68BBE
:10031600E511F0250DF50DE510350CF50CC3E50FCF
:100326009511F50FE50E9510F50E02026E90E6B8E2
:10033600E0644060030203CCE50F450E7003020340
:10034600CCE490E68AF090E68BF090E6A0E020E11F
:10035600F990E68BE0751000F51190E6B9E0B4A3CC
:1003660036E4F512F513C3E5139511E51295105011
:100376003774402513F58274E73512F583E0FFE5FF
:100386000D2513F582E50C3512F583EFF00513E51F
:100396001370D3051280CFAD117AE779407F40AB59
:1003A60007AF0DAE0C120BF5E511250DF50DE51099
:1003B600350CF50CC3E50F9511F50FE50E9510F507
:0703C6000E02033ED322C327
:0103CD00220D
:100D3300C0E0C083C08290E6B5E04401F0D2015325
:0F0D430091EF90E65D7401F0D082D083D0E03262
:100DA200C0E0C083C0825391EF90E65D7404F0D03E
:060DB20082D083D0E03284
:100DB800C0E0C083C0825391EF90E65D7402F0D02A
:060DC80082D083D0E0326E
:1007C500C0E0C083C08290E680E030E70E85212539
:1007D500852226852927852A28800C852925852A8D
:1007E500268521278522285391EF90E65D7410F028
:0707F500D082D083D0E03276
:100D8A00C0E0C083C082D2035391EF90E65D74083D
:080D9A00F0D082D083D0E032DA
:100B8800C0E0C083C08290E680E030E70E85212572
:100B9800852226852927852A28800C852925852AC6
:100BA800268521278522285391EF90E65D7420F051
:070BB800D082D083D0E032AF
:01003200329B
:01004200328B
:01005200327B
:010E180032A7
:010E190032A6
:010E1A0032A5
:010E1B0032A4
:010E1C0032A3
:010E1D0032A2
:010E1E0032A1
:010E1F0032A0
:010E2000329F
:010E2100329E
:010E2200329D
:010E2300329C
:010E2400329B
:010E2500329A
:010E26003299
:010E27003298
:010E28003297
:010E29003296
:010E2A003295
:010E2B003294
:010E2C003293
:010E2D003292
:010E2E003291
:010E2F003290
:010E3000328F
:010E3100328E
:010E3200328D
:010E3300328C
:010E3400328B
:010E3500328A
:010E36003289
:010E37003288
:010E38003287
:040B4900AA06AC0547
:100B4D00E4FD7E000DEE2400F582E43400F583EA29
:100B5D00F00E0D74002EF582E43400F583EFF00DE8
:100B6D0074002402F582E43400F583ECF07A007B06
:0B0B7D0000AF32120D6EAF32020BBF52
:0A0BF5008E148F158D168A178B18C9
:100BFF00E4F519E519C3951650200515E515AE1442
:100C0F007002051414FFE5182519F582E43517F560
:0A0C1F0083E0FD120B49051980D98E
:010C290022A8
:0A0ABB008E148F158D168A178B1804
:100AC500E4FDF519E5356012E514FF7E000DEE2411
:100AD50000F582E43400F583EFF0AE050D74002EC9
:100AE500F582E43400F583E515F07A007B00AF323A
:0E0AF500120D6EAB18AA17AD16AF32020D52DD
:100C900090E682E030E004E020E60B90E682E0306F
:100CA000E119E030E71590E680E04401F07F147E22
:0C0CB00000120B0390E680E054FEF022DE
:100D0E0090E682E044C0F090E681F0438701000057
:040D1E0000000022AF
:1000030030040990E680E0440AF0800790E680E03F
:100013004408F07FDC7E05120B0390E65D74FFF06D
:0F00230090E65FF05391EF90E680E054F7F02203
:080E0200E4F51FD2E9D2AF2292
:100BBF0090E678E020E6F9C2E990E678E04480F02C
:100BCF00EF25E090E679F090E678E030E0F990E6F6
:100BDF0078E04440F090E678E020E6F990E678E09F
:060BEF0030E1D6D2E9223C
:100C5E00A90790E678E020E6F9E51F702390E67884
:100C6E00E04480F0E925E090E679F08D1AAF03A913
:100C7E0007751B018A1C891DE4F51E751F01D32201
:020C8E00C3227F
:100C2A00A90790E678E020E6F9E51F702590E678B6
:100C3A00E04480F0E925E0440190E679F08D1AAFAE
:100C4A0003A907751B018A1C891DE4F51E751F037C
:040C5A00D322C322BC
:03004B000205F3B8
:1005F300C0E0C083C082C085C084C086758600C049
:10060300D075D000C000C001C002C003C006C0073F
:1006130090E678E030E206751F060206DD90E67884
:10062300E020E10CE51F64026006751F070206DD8A
:10063300E51F24FE605F14603624FE70030206CEBD
:1006430024FC70030206DA240860030206DDAB1BF8
:10065300AA1CA91DAF1E051E8F827583001206FBFF
:1006630090E679F0E51E651A7070751F05806B9032
:10067300E679E0AB1BAA1CA91DAE1E8E8275830012
:10068300120728751F02E51A6401704E90E678E0A0
:100693004420F08045E51A24FEB51E0790E678E075
:1006A3004420F0E51A14B51E0A90E678E04440F0C1
:1006B300751F0090E679E0AB1BAA1CA91DAE1E8E28
:1006C30082758300120728051E800F90E678E044A8
:1006D30040F0751F008003751F005391DFD007D0D2
:1006E30006D003D002D001D000D0D0D086D084D0A1
:0806F30085D082D083D0E032F3
:020CBC00A90786
:100CBE00AE2DAF2E8F828E83A3E064037017AD012D
:100CCE0019ED7001228F828E83E07C002FFDEC3EA9
:090CDE00FEAF0580DF7E007F00FF
:010CE70022EA
:100D5200120C2AE51F24FA600E146006240770F3B1
:0C0D6200D322E4F51FD322E4F51FD322B6
:100D6E00120C5EE51F24FA600E146006240770F361
:0C0D7E00D322E4F51FD322E4F51FD3229A
:100B03008E0C8F0D90E600E054187012E50D240151
:100B1300FFE4350CC313F50CEF13F50D801590E6C8
:100B230000E05418FFBF100BE50D25E0F50DE50CB3
:100B330033F50CE50D150DAE0C7002150C4E60056A
:060B4300120D2280EE22DB
:100D22007400F58690FDA57C05A3E582458370F9E4
:010D3200229E
:03004300020800B0
:03005300020800A0
:10080000020D3300020DB800020DA200020D8A0095
:100810000207C500020B88000200320002004200FD
:1008200002005200020E1800020E1900020E1A00F9
:10083000020E1B00020E1C00020E1D00020E1E0006
:10084000020E1F0002004200020E2000020E2100D4
:10085000020E2200020E2300020E2400020E2500CA
:10086000020E260002004200020042000200420086
:10087000020E2700020E2800020E2900020E2A0096
:10088000020E2B00020E2C00020E2D00020E2E0076
:10089000020E2F00020E3000020E3100020E320056
:1008A000020E3300020E3400020E3500020E360036
:0808B000020E3700020E3800B1
:030000000209E40E
:0C09E400787FE4F6D8FD758135020A2BFF
:1006FB00BB010CE58229F582E5833AF583E02250B4
:10070B0006E92582F8E622BBFE06E92582F8E222FD
:0D071B00E58229F582E5833AF583E4932217
:10072800F8BB010DE58229F582E5833AF583E8F007
:10073800225006E92582C8F622BBFE05E92582C8B3
:02074800F2229B
:10074A00BC000BBE0029EF8DF084FFADF022E4CC93
:10075A00F875F008EF2FFFEE33FEEC33FCEE9DEC5C
:10076A00984005FCEE9DFE0FD5F0E9E4CEFD22EDA2
:10077A00F8F5F0EE8420D21CFEADF075F008EF2FEC
:10078A00FFED33FD4007985006D5F0F222C398FDDD
:05079A000FD5F0EA227A
:10079F00D083D082F8E4937012740193700DA3A3E9
:1007AF0093F8740193F5828883E4737402936860FD
:0607BF00EFA3A3A380DFFD
:1009F000020956E493A3F8E493A34003F68001F2BE
:100A000008DFF48029E493A3F85407240CC8C33307
:100A1000C4540F4420C8834004F456800146F6DFD6
:100A2000E4800B0102040810204080900046E47E20
:100A3000019360BCA3FF543F30E509541FFEE493CB
:100A4000A360010ECF54C025E060A840B8E493A392
:100A5000FAE493A3F8E493A3C8C582C8CAC583CABD
:100A6000F0A3C8C582C8CAC583CADFE9DEE780BE75
:01004A0000B5
:00000001FF
